:103ECE000F580F4E0F430F380F2D0F210F140F07E2
:103EDE000EF90EEB0EDC0ECC0EBC0EAB0E9A0E8750
:103EEE000E750E610E4D0E380E220E0C0DF40DDCFD
:103EFE000DC40DAA0D900D750D5A0D3E0D210D031D
:103F0E000CE40CC50CA50C850C640C420C200BFDAE
:103F1E000BD90BB50B900B6B0B460B200AF90AD382
:103F2E000AAC0A840A5D0A350A0D09E409BC099334
:103F3E00096B0942091A08F108C808A00878085048
:103F4E000828080007D807B1078A0764073E071834
:103F5E0006F206CD06A906840661063E061B05F886
:103F6E0005D705B50595057405550535051704F9ED
:103F7E0004DB04BE04A20486046A044F0435041B49
:103F8E00040203E903D103B903A2038B0375035F94
:103F9E00034A03350321030D02FA02E702D502C3D9
:103FAE0002B102A0028F027F026F025F0250024135
:103FBE00023302250217020A01FD01F001E301D7C7
:103FCE0001CC01C001B501AA019F0195018B0181B0
:103FDE000178016E0165015C0154014B0143013B07
:103FEE000133012C0125011D0116011001090102E9
:103FFE0000FC00F600F000EA00E500DF00DA00D475
:10400E0000CF00CA00C600C100BC00B800B300AFAC
:10401E0000AB00A700A3009F009B009800940091A6
:10402E00008D008A00870084008100010C010105CB
:10403E0002011E030A9604013205030306006407FB
:10404E00010108000009015A0E01010F00011200C2
:10405E006413010114013C1501FA1664FA17FFFFEF
:10406E001D00072000072400022701012F013C300C
:10407E00020232010335FFFF3603073CFFFF3DFF0F
:10408E00FF180002191E461A00021B00022D32C82C
:06409E002E0001FAFAFAFF
:10004800900786E0FEA3E0FF7457BE0010D39F40E0
:100058000C90403812001EE493F5998012900786A0
:10006800E0FEA3E0FF90403812001EE493F599905B
:10007800078612000E900786E0FEA3E0FF746C6FFF
:100088004E700375130022900072E0B402087401E8
:10009800900072F0D20F90013AE090002AF090019F
:1000A8003BE090002BF090013CE090002CF0A20A7D
:1000B800B3401690013AE0700C90013BE070069056
:1000C800013CE060028002C20A90013AE0B4300FBD
:1000D80090013BE0B4470890013CE0643B6002803B
:1000E80004D20B8002C20BE559B40102800302025C
:1000F80011900057E0F567900062E0F569900063A1
:10010800E0F56A900074E0F56B90007AE0900029C1
:10011800F090007CE0F56690007DE0F56890008046
:10012800E0F565900081E0F564900090E090004172
:10013800F0900091E0900042F0900092E09000432F
:10014800F0900093E0900044F0900094E090004517
:10015800F0900095E0900046F0900096E0900047FF
:10016800F0900097E0900048F0900099E0900033FC
:10017800F090009AE0900034F090009BE0900035F9
:10018800F090009CE0900036F0900079E0B4011700
:1001980090000A740FF0A374FFF090000CE4F0A331
:1001A800F07402900079F0900079E0B4035990005F
:1001B8000CE0FEA3E0FF90000AE0FCA3E0FD1200C3
:1001C80003741012420474081241F6EF900026F0EE
:1001D800EF700674FF900026F07400900079F0909C
:1001E800000BE0900027F090000AE0900028F090C3
:1001F8000026E0900789F0900027E090078AF090A9
:100208000028E090078BF0803F900081E070067531
:100218005901756400A20AB3402E90013AE090009B
:100228002AF090013BE090002BF090013CE0900018
:100238002CF090002AE0700C90002BE070069000E3
:100248002CE060028002C20AE5677003756702E568
:100258006970037569027E837FC2E5678E048F0526
:10026800FF1241E68C398D3AE56A75F0FAA4FFAEC3
:10027800F0E5698E048F05FF1241E68C3D8D3E90B6
:10028800004FE0F56190004DE0FE900069E0B50692
:100298001890004CE0FE900068E0B5060C90004B0A
:1002A800E0FE900059E06E606F900069E070069083
:1002B8000068E060067400900059F0900069E0B4AE
:1002C80002089000497401F08005900049E4F0901C
:1002D8000068E0B4020890004A7401F080059000BC
:1002E8004AE4F0900068E0600690004AE06002800E
:1002F800057561048003756105E55AB55902D20F89
:10030800900068E090004CF0900069E090004DF09B
:10031800900059E090004BF0740190009EF074003A
:1003280090009FF074019000A0F074009000A1F07C
:1003380074019000A2F074009000A3F07400900083
:10034800A4F074009000A5F074019000A6F0740069
:100358009000A7F074019000A8F074019000A9F033
:1003680074019000AAF074009000ABF07401900042
:10037800ACF074009000ADF074019000AEF0740021
:100388009000AFF074019000B0F074009000B1F0EC
:1003980074009000B2F07401900362F0740090034E
:1003A80063F07400900364F07401900365F07401C5
:1003B800900366F07401900367F07400900368F08E
:1003C80074019003A2F074019003A3F074009003E9
:1003D800A4F074009003A5F074019003A6F07401D2
:1003E8009003A7F074009003A8F074009003E2F063
:1003F80074019003E3F074009003E4F07401900337
:10040800E5F074019003E6F074009003E7F07400DF
:100418009003E8F07400900422F07401900423F033
:100428007400900424F07400900425F07400900483
:1004380026F07400900427F07400900428F07400EB
:10044800900462F07400900463F07400900464F007
:100458007401900465F07400900466F074009004D0
:1004680067F07400900468F022E5B554F7F5B5C25A
:10047800A1C293C294C291C292757000E5B554FDB1
:10048800F5B5C207E5B554FBF5B5755105E5510459
:10049800F55290004FE0F561900025E4F0C209E5BF
:1004A800B554FEF5B522750A00750900AE09AF0A04
:1004B8007457BE00039F500302056B90403812002A
:1004C8001EE49390004E12421C0FBF00010EE0FC88
:1004D80090403812001EECFEE493FFEEC39F5026B6
:1004E800AE09AF0A0FBF00010E90403812001EAED1
:1004F80009AF0AE493FC90403812001EE493900080
:100508004E12421CECF0AE09AF0A90403812001EA1
:10051800E49390004E12421CE0FC90403A12001EF8
:10052800ECFCE493FDECD39D401990403A12001E78
:10053800E493FC90403812001EE49390004E12425F
:100548001CECF0AE09AF0A74022FFF50010E8E09A1
:100558008F0A780A740126F6500418E436F6400328
:100568000204B422750A00750900AE09AF0A7415B1
:10057800BE00039F500302063990408F12001EE40C
:100588009390004E12421C0FBF00010EE0FC9040F9
:100598008F12001EECFEE493FFEEC39F5026AE09B7
:1005A800AF0A0FBF00010E90408F12001EAE09AFB8
:1005B8000AE493FC90408F12001EE49390004E12C0
:1005C800421CECF0AE09AF0A90408F12001EE49373
:1005D80090004E12421CE0FC90409112001EECFC70
:1005E800E493FDECD39D401990409112001EE493D2
:1005F800FC90408F12001EE49390004E12421CECB7
:10060800F0AE09AF0A740F6F4E7006750A157509BA
:1006180000AE09AF0A74022FFF50010E8E098F0A2F
:10062800780A740126F6500418E436F640030205E9
:100638007222054D22054C22054EC2CF2290F800A9
:10064800E4936406600280FE75840175A70075FF57
:1006580080900788E4F075C91075A70F75A1C77554
:10066800A70075D90075CEFF75A70F75F1FE75F255
:10067800FF75F33775F47875A4BA75A5FF75A607E5
:1006880075AE0075AFFF75D48175D5FF75D6FF754A
:10069800D7FFE5B554EFF5B5E5B554DFF5B5C28735
:1006A800E5B554BFF5B5E5B5547FF5B575A7007543
:1006B800A20175A14775F80975BC0175BE0475BD21
:1006C8006C75BE0775BDA075BE0875BD0175BC000B
:1006D80075BB1875BC2075BA0875E88075D1137597
:1006E800A70F75E10575E20075C740759700759706
:1006F80080740A1241D67597C0E59754207002801D
:10070800F8758F0275A700D2AF75980075A90C759A
:10071800A70F75AB4375ADFB75AC1E75A700758942
:1007280011758E00758C00758A00D2A9D28C758DD2
:1007380000758B00D2ABD28E75CD0075CC0075CA12
:100748000075CB00D2ADC2CFD2CA759104759200A4
:100758007593CD75EF0675D94075CF01900786E47E
:10076800F0A3F0751300751400C299D20A74C8F585
:10077800187517001227F775A70FE5FB90001AF0F8
:10078800E5FA90001BF0E5F990001CF075A70090C1
:10079800F800E493F50812292E122E68900789E0D4
:1007A800900026F090078AE0900027F090078BE0F1
:1007B800900028F090078CE0900029F090078DE0D9
:1007C800F56790078EE0F56990078FE0F56A900766
:1007D80090E0F56B900791E0F566900792E0F56878
:1007E800900793E0F565900794E0F564900795E02D
:1007F80090002AF0900796E090002BF0900797E081
:1008080090002CF0900798E0900041F0900799E054
:10081800900042F090079AE0900043F090079BE028
:10082800900044F090079CE0900045F090079DE010
:10083800900046F090079EE0900047F090079FE0F8
:10084800900048F09007A0E0900033F09007A1E0F6
:10085800900034F09007A2E0900035F09007A3E0F4
:10086800900036F07400900082F090013AE0700C2D
:1008780090013BE0700690013CE060028004C20AEF
:100888008002D20A90F807E493900021F0900021AA
:10089800E0440A900021F0900021E054FE900021ED
:1008A800F07406900012F07402900013F090F802B1
:1008B800E493900014F07403900015F07403900012
:1008C80016F0741E900017F07405900018F0740468
:1008D800900019F090F804E49390001DF0740090D3
:1008E800001EF090F805E49390001FF090F806E4DD
:1008F80093900020F074FF900022F0745A90012524
:10090800F07446900126F07420900127F074359019
:100918000128F07448900129F0745090012AF0746D
:100928003290012BF0743490012CF0742090012D3A
:10093800F0743590012EF0745390012FF07470907C
:100948000130F07465900131F07465900132F074F3
:1009580064900133F090007AE0D39401400674006B
:1009680090007AF0755901755A01740390004CF0A3
:1009780012008F1204AE12056C122823E5B554FE3E
:10098800F5B5900025E4F0900786E4F0A3F075240F
:1009980000752300754800752A00752900754900FF
:1009A800753200753100754A00755400755500752B
:1009B8005B0075510575520175343C7533007572CD
:1009C800007571007573CD75560075570075580020
:1009D800754300754400754500754600755C0075E3
:1009E8004700754200754100900006E4F0A3F090BE
:1009F8000008E4F0A3F0755F0075600090000E74C5
:100A0800FDF0A374E8F0900023E4F07464900024EF
:100A1800F0C200D201C202D203754D00756E00C249
:100A280097C2A0C296C295C2A2C20F7E017F009053
:100A38000028E0124204900027E02FFF50010E909A
:100A4800000AEEF0A3EFF0900026E0700674FF9025
:100A58000026F090000AE0FEA3E0FFEFD394FFEE3B
:100A6800940F400790000AE4F0A3F074009000711E
:100A7800F07400900079F07400900082F074009097
:100A8800008DF074009000B4F0E568700375680498
:100A9800743A90074EF074FD90074FF0900414E0FC
:100AA800900454F0D2B0D2B7D2A7D2A6D2B1D2A372
:100AB800C207A2B6B39204A2B3B39205D29CD2ECF9
:100AC80075CF01A298B34005C2981231CCE51360E6
:100AD80006A299B3B340028005C299123742E514C1
:100AE80064016005E514B4040280D5E54DD394058E
:100AF800400CE55BC394C85002055B754D00E57377
:100B0800C394F0501A787112003FAE71AF72EFD3F0
:100B180094E8EE940340080573757200757100C27D
:100B28008E7E047F00E54C124204E58D75F004A426
:100B3800FDACF0EF2DFDEE3CFCE58B75F04084FF3D
:100B48007E00ED2FFFEC3EFE8E258F26D28EA2B6BC
:100B5800300401B35003020C82A2B6300401B35032
:100B680003020C82A2B6405A0554E5B54401F5B516
:100B7800900024E4F0E554D3956740447C837DC21B
:100B88001240A48E238F24E5482FFF50010E7401D4
:100B98001241F68E238F24852448755401C28E7520
:100BA8008D00758B00754C00D28E7403BE00039FB8
:100BB80050069000257401F0E543B4060375430020
:100BC800D204A2B6B35003020C82C20490006BE0B8
:100BD8006018123883A200B34008E5B54408F5B59B
:100BE8008006E5B554F7F5B58002C20090006EE0C6
:100BF80060101239D8A202B34004D2A18002C2A167
:100C08008002C2A1A207B34004D2968002C2969085
:100C18000059E06004D2958002C29590004AE0B481
:100C28000104D2978002C297900049E0B40104D22F
:100C3800A08002C2A0A209B34004D2A28002C2A22C
:100C4800900018E0FE900014E0C39E400990001444
:100C5800E0D39408400974FB900023F012047190CB
:100C6800001DE0601590001DE0FE900017E06E602A
:100C78000974FE900023F0120471C2CA7E017F003D
:100C8800E54E124204E5CD2FFF50010E8E278F2826
:100C9800D2CAE566B4014890000EE0FCA3E0FDEF7F
:100CA800C39DEE9C4039B208E52A45296013A20885
:100CB800B34008E5B54404F5B58006E5B554FBF541
:100CC800B590000EE0FEA3E0FF900010E0FCA3E06A
:100CD800FDEF2DFDEE3CFC90000EECF0A3EDF0A234
:100CE800B3300501B35003020DC7A2B3300501B3F9
:100CF8005003020DC7A2B35003020DC00555E5B558
:100D08004401F5B5900024E4F0E555D39569500306
:100D1800020DBE7CEA7D60AE27AF281240A48E2962
:100D28008F2AE56A12420474FF8E048F05FF124170
:100D3800E68C298D2AE5492DFD50010C74018C069D
:100D48008D071241F68E298F2A852A49A209B340B8
:100D5800157464124204900067E08E048F05FF1238
:100D680041E68C298D2A75550190000EE0FEA3E01E
:100D7800FFAC27AD2812000390000EEEF0A3EFF0B1
:100D8800E568FF1241E6740AFF1241E690007BE035
:100D98008C068D0712420474148E048F05FF1241CD
:100DA800E6900010ECF0A3EDF0C2CA75CD0075CC4A
:100DB80000754E00D2CAD205A2B3B34002C2059054
:100DC8000025E0B40107E556C3940640030213DF8B
:100DD800E56E9027D6F8282873900059E0C394024E
:100DE8004003020F35E551D394015003020F35E556
:100DF8005175F040A4FFAEF090031212001EE0C33C
:100E080095455018E55175F040A4FFAEF0900311D8
:100E180012001EE0F52E752D00020F35E55175F014
:100E280040A4FFAEF090031012001EE0C3954540A9
:100E380003020ED1E55175F040A4FFAEF090031106
:100E480012001EE55175F040A4FFAEF0E0FC9003DF
:100E58000F12001EECFEE0FFEEC39FFEE5518E046C
:100E680075F040A4FFAEF090031012001EE0F404E9
:100E780025458C0088F0A4FFAEF0E5518F048E055F
:100E880075F040A4FFAEF090031212001EE55175F4
:100E9800F040A4FFAEF0E0FA90031012001EEAFE44
:100EA800E0FFEEC39FFECDCCCD8E071241E6E551A3
:100EB80075F040A4FFAEF090030F12001EE02DFD68
:100EC80050010C8C2D8D2E8064E55175F040A4FFE7
:100ED800AEF090030F12001EE55175F040A4FFAE6E
:100EE800F0E0FC90030E12001EECFEE0FFEEC39F44
:100EF8008545F0A4FFAEF0E5518F048E0575F040EE
:100F0800A4FFAEF090031012001EE0FECDCCCD8EF3
:100F1800071241E6E55175F040A4FFAEF090030ECC
:100F280012001EE02DFD50010C8C2D8D2E756E01CA
:100F38000213DF900059E0C3940240030210E990C5
:100F4800004FE0D395515003021091E55175F040E0
:100F5800A4FFAEF090031812001EE0C39545501888
:100F6800E55175F040A4FFAEF090031712001EE0A3
:100F7800F52C752B00021091E55175F040A4FFAED9
:100F8800F090031612001EE0C39545400302102D91
:100F9800E55175F040A4FFAEF090031712001EE56E
:100FA8005175F040A4FFAEF0E0FC90031512001E4E
:100FB800ECFEE0FFEEC39FFEE5518E0475F040A401
:100FC800FFAEF090031612001EE0F40425458C00D5
:100FD80088F0A4FFAEF0E5518F048E0575F040A4AB
:100FE800FFAEF090031812001EE55175F040A4FF03
:100FF800AEF0E0FA90031612001EEAFEE0FFEEC320
:101008009FFECDCCCD8E071241E6E55175F040A488
:10101800FFAEF090031512001EE02DFD50010C8C60
:101028002B8D2C8064E55175F040A4FFAEF0900341
:101038001512001EE55175F040A4FFAEF0E0FC90DB
:10104800031412001EECFEE0FFEEC39F8545F0A4DA
:10105800FFAEF0E5518F048E0575F040A4FFAEF0A9
:1010680090031612001EE0FECDCCCD8E071241E68D
:10107800E55175F040A4FFAEF090031412001EE095
:101088002DFD50010C8C2B8D2CE551B40123E5610D
:10109800D39401401CE55604D395514014E545C34B
:1010A8009405500D90035FE0A829B80006952A40E2
:1010B800028003755102E551B5612290004FE0D3DB
:1010C80095514019E55175F040A4FFAEF090031713
:1010D80012001EE0A823B8000695244002800205ED
:1010E80061756E020213DF900059E0B4022AE551DF
:1010F80075F040A4FFAEF090031712001EE0F52C27
:10110800752B00E55175F040A4FFAEF090030E1268
:10111800001EE0F52E752D00900059E0B4030F90E5
:101128000051E0F52C752B00752E00752D00756E9D
:10113800030213DFE55175F040A4FFAEF0900320E1
:1011480012001EE0C3955B4003021215900049E0AF
:101158007036E551D394014029AE23AF24AC2DADB0
:101168002EEDD39FEC9E401AE55175F040A4FFAEDA
:10117800F090031E12001EE0A829B80005D3952A96
:101188005002800215518034E551D394024029AEB3
:1011980023AF24AC2DAD2EEDD39FEC9E401AE55124
:1011A80075F040A4FFAEF090031E12001EE0A829BF
:1011B800B80005D3952A500280021551E551B55261
:1011C80037E551C395615030E55604D39551402811
:1011D800AE23AF24AC2BAD2CEFD39DEE9C4019E58C
:1011E8005175F040A4FFAEF090031F12001EE0A856
:1011F80029B80006952A400280020551E5B554FD3C
:10120800F5B5E55165526005C207755B00756E045A
:101218000213DFE55175F040A4FFAEF090031A12F7
:10122800001EE0B40117E55175F040A4FFAEF09040
:10123800032012001EE0240AC3955B40030212EB50
:10124800753064752F00A207B3500B900060E0243E
:1012580005C3954540030212EBE55175F040A4FF24
:10126800AEF090031D12001EE0C395454064E551A1
:1012780075F040A4FFAEF090031C12001EE55175F6
:10128800F040A4FFAEF0E0FC90031B12001EECFE41
:10129800E0FFEEC39F8545F0A4FFAEF0E5518F0453
:1012A8008E0575F040A4FFAEF090031D12001EE0FD
:1012B800FECDCCCD8E071241E6E55175F040A4FF76
:1012C800AEF090031B12001EE02DFD50010C8C2F78
:1012D8008D30AE23AF24AC2FAD30EFD39DEE9C40C4
:1012E80002D207756E050213DFE551B401099000BB
:1012F80059E0C3940240030213BF900358E0D3950A
:101308004550030213BF900356E0C39545504090E3
:101318000357E0FE900355E0F4042EFE900356E0D8
:10132800F40425458E0088F0A4FFAEF0900358E041
:10133800FC900356E0F4042C8E048F05FF1241E65E
:10134800900355E02DFD50010C8C2B8D2C802C909A
:101358000355E0FE900354E0F4042E8545F0A4FF05
:10136800AEF0900356E08E048F05FF1241E690031D
:1013780054E02DFD50010C8C2B8D2CE551C395614B
:101388005030E55604D395514028AE23AF24AC2BFA
:10139800AD2CEFD39DEE9C4019E55175F040A4FFAC
:1013A800AEF090031F12001EE0A829B80006952A87
:1013B80040028003755102900049E0B40106E551EE
:1013C800640160028003755102E55165526005C2EF
:0713D80007755B00756E0054
:1027D600020DE1020F3B0210EF02113C02121B0236
:0227E60012F1EE
:1013DF00900050E02402A823B80007D395244002C0
:1013EF00C207900025E0B40109900059E0C39403AF
:1013FF004003021567900049E060030214B6E551FF
:10140F00D394014034E55175F040A4FFAEF0900342
:10141F001412001EE0A823B8001FD39524401AE52C
:10142F005175F040A4FFAEF090031F12001EE0A80C
:10143F0029B80005D3952A500280021551E551D3E2
:10144F009401402FE55175F040A4FFAEF0900312C8
:10145F0012001EE0C39545501AE55175F040A4FFE8
:10146F00AEF090031E12001EE0A829B80005D39518
:10147F002A500280021551E551D394014022E556BE
:10148F0004C39551501AE55175F040A4FFAEF0908A
:10149F00031E12001EE0A829B80005D3952A50029A
:1014AF008002155102155CE551D394024034E55189
:1014BF0075F040A4FFAEF090031412001EE0A823B5
:1014CF00B8001FD39524401AE55175F040A4FFAE24
:1014DF00F090031F12001EE0A829B80005D3952A2B
:1014EF00500280021551E551D39402402FE55175FA
:1014FF00F040A4FFAEF090031212001EE0C395451A
:10150F00501AE55175F040A4FFAEF090031E120083
:10151F001EE0A829B80005D3952A50028002155164
:10152F00E551D394024022E55604C39551501AE574
:10153F005175F040A4FFAEF090031E12001EE0A8FC
:10154F0029B80005D3952A500280021551E551653F
:10155F00526005C207755B00900060E0D39545505F
:10156F0009900054E0C395455002C207900059E01E
:10157F0070030217CCA2A5B34008A2A4B340030284
:10158F0017B5AE35AF367441D39F749C9E40057826
:10159F003512003FAE35AF36EFB48806EEB4130206
:1015AF008003021792A2A55003021655900059E02E
:1015BF00B4010B90004FE0D395614002056190009C
:1015CF0059E0B40254E55175F040A4FFAEF090031A
:1015DF002012001EE0C3955B503F90004FE0D39563
:1015EF00514021E55604D395514019E55175F0400E
:1015FF00A4FFAEF090031412001EE0A823B800065B
:10160F00952440028002055190004FE0F561E551AD
:10161F0065526005C207755B00900059E0B4032660
:10162F0090004FE0D395514008E55604D3955150A3
:10163F00028002055190004FE0F561E5516552605F
:10164F0005C207755B00A2A45003021792900059C0
:10165F00E0B4016E900049E07035E551D39401403C
:10166F0029E55175F040A4FFAEF090031E12001E45
:10167F00E0A829B8000FD3952A400A1551755B00D1
:10168F00855161800385516180037561018033E568
:10169F0051D394024029E55175F040A4FFAEF0906C
:1016AF00031E12001EE0A829B8000FD3952A400A86
:1016BF001551755B008551618003855161800375FC
:1016CF006102900059E0D394015003021786E5514F
:1016DF0075F040A4FFAEF090032012001EE0C395FA
:1016EF005B4003021786900049E07041E551D394A7
:1016FF00014034E55175F040A4FFAEF09003111294
:10170F00001EE0A823B8001FD39524401AE5517599
:10171F00F040A4FFAEF090031E12001EE0A829B8FF
:10172F000005D3952A500280021551803FE551D311
:10173F0094024034E55175F040A4FFAEF0900311D0
:10174F0012001EE0A823B8001FD39524401AE551BC
:10175F0075F040A4FFAEF090031E12001EE0A82902
:10176F00B80005D3952A500280021551E5516552F4
:10177F006005C207755B00E556B40704055F80037B
:10178F00755F00E564B4010EAE35AF36EF6440709F
:10179F0005EE649C6002800EA2A54003755901A25C
:1017AF00A44003755902A2A5B3B35006A2A4B3B3C4
:1017BF00400280067536007535000218BAA2A5B32F
:1017CF004008A2A4B340030218A6AE35AF36744149
:1017DF00D39F749C9E4005783512003FAE35AF36CF
:1017EF00EFB48806EEB4130280030218A6A2A54038
:1017FF006F900068E0605A90004AE0B401079000D3
:10180F004AE4F0800690004A7401F090004AE070BC
:10181F0005756104800375610590004AE0B4010409
:10182F00D2978002C297E551B4051AE55175F04081
:10183F00A4FFAEF090031E12001EE0A829B8000509
:10184F00D3952A50028008755104C207755B00803A
:10185F0003756105E556B40704055F8003755F00E6
:10186F00A2A44033900069E06021900049E0B401E8
:10187F0007900049E4F080069000497401F0900051
:10188F0049E0B40104D2A08002C2A0E556B4070417
:10189F00055F8003755F00A2A5B3B35006A2A4B382
:1018AF00B340028006753600753500E559655A60FC
:1018BF0006900082E06003021A42C29C7514007504
:1018CF001300C2CAE5599027E8F82828738012122E
:1018DF002E68800D122F41800812301A80031230AB
:0118EF00F305
:0F27E8000218DC0218DE0218E30218E80218EDEE
:1018F000900029E090007AF0E567900057F0E569E4
:10190000900062F0E56A900063F0E56B900074F07F
:10191000E56690007CF0E56890007DF0E56590005C
:1019200080F0E564900081F090002AE090013AF0A8
:1019300090002BE090013BF090002CE090013CF0F7
:10194000900041E0900090F0900042E0900091F013
:10195000900043E0900092F0900044E0900093F0FB
:10196000900045E0900094F0900046E0900095F0E3
:10197000900047E0900096F0900048E0900097F0CB
:10198000900033E0900099F0900034E090009AF0DD
:10199000900035E090009BF0900036E090009CF0C5
:1019A0007400900082F0745A900125F07446900102
:1019B00026F07420900127F07435900128F07448C7
:1019C000900129F0745090012AF0743290012BF0AC
:1019D000743490012CF0742090012DF07435900136
:1019E0002EF0745390012FF07470900130F07465F4
:1019F000900131F07465900132F07464900133F01D
:101A00009003D4E0900414F0743A90074EF074FD03
:101A100090074FF012008F900004E4F0A3F09000C4
:101A2000067475F0A37430F09000087475F0A37418
:101A300030F085595AD2CA754C00D29C741B900064
:101A400023F0900025E0B401028003021EA1E556B8
:101A5000C394065005E551B55203021B31C207E598
:101A60005175F040A4FFAEF090032212001EE0304A
:101A7000E003D38001C3B34008E5B54410F5B58059
:101A800006E5B554EFF5B5E55175F040A4FFAEF0AD
:101A900090032312001EE030E003D38001C3B34063
:101AA00008E5B54420F5B58006E5B554DFF5B5E5A4
:101AB0005175F040A4FFAEF090032412001EE030F8
:101AC000E003D38001C39287E55175F040A4FFAED7
:101AD000F090032512001EE030E003D38001C39292
:101AE0000CE55175F040A4FFAEF090032612001EE5
:101AF000E030E003D38001C3920DE55175F040A4BE
:101B0000FFAEF090032712001EE030E003D3800107
:101B1000C3920E855152AE29AF2A7405BE00039FB1
:101B20005007E545D3940550028006E5B54402F51B
:101B3000B5E556D394055003021DA0C207E551D365
:101B400094015003021C34E55175F040A4FFAEF03F
:101B500090031E12001EE0A829B80007D3952A4062
:101B6000021551E55165527003021C31E55175F0C3
:101B700040A4FFAEF090032212001EE030E003D339
:101B80008001C3B34008E5B54410F5B58006E5B55E
:101B900054EFF5B5E55175F040A4FFAEF090032386
:101BA00012001EE030E003D38001C3B34008E5B566
:101BB0004420F5B58006E5B554DFF5B5E55175F07F
:101BC00040A4FFAEF090032412001EE030E003D3E7
:101BD0008001C39287AE29AF2A7405BE00039F50CF
:101BE00002D287E55175F040A4FFAEF090032512B4
:101BF000001EE030E003D38001C3920CE55175F084
:101C000040A4FFAEF090032612001EE030E003D3A4
:101C10008001C3920DE55175F040A4FFAEF0900332
:101C20002712001EE030E003D38001C3920E8551DD
:101C300052021DA0E556B406709000ACE030E008FA
:101C4000E5B54410F5B58006E5B554EFF5B590005F
:101C5000ADE030E008E5B54420F5B58006E5B554C3
:101C6000DFF5B59000AEE030E003D38001C392878A
:101C70009000AFE030E003D38001C3920CE55BD36A
:101C800094034002D20C9000B0E030E003D3800116
:101C9000C3920D9000B1E030E003D38001C3920EF7
:101CA000E55BD394034002D20EE556B4077D900065
:101CB000A5E030E008E5B54410F5B58006E5B5547B
:101CC000EFF5B59000A6E030E008E5B54420F5B5A5
:101CD0008006E5B554DFF5B5AE29AF2A7406BE001F
:101CE00011D39F400D9000A7E030E003D38001C3E3
:101CF00092879000A8E030E003D38001C3920CE506
:101D00005BD394034002C20C9000A9E030E003D3FF
:101D10008001C3920D9000AAE030E003D38001C39C
:101D2000920EE55BD394034002C20EE556B40870F0
:101D300090009EE030E008E5B54410F5B58006E57A
:101D4000B554EFF5B590009FE030E008E5B54420CC
:101D5000F5B58006E5B554DFF5B59000A0E030E0BC
:101D600003D38001C392879000A1E030E003D380C9
:101D700001C3920CE55BD394034002D20C9000A205
:101D8000E030E003D38001C3920D9000A3E030E087
:101D900003D38001C3920EE55BD394034002D20EBD
:101DA000E551B40107E556C3940640028012E55B95
:101DB000D394034002C20CE55BD394034002C20EED
:101DC000900072E06058E54575F00284FF7E009057
:101DD000014E12001EE0F55DE54775F00A84FF7EB6
:101DE0000090024E12001EE0F55EE55D255ED39484
:101DF00064400BE55D255EC39464F55D8003755D0D
:101E000000E55D75F00284FF7E008F5DEFC39433C3
:101E10005007EF24CDF55D8003755DFF801CE5451F
:101E200075F00284FF7E0090014E12001EE075F0F6
:101E30000284FF7E00EF24CDF55DE595C3955D40FE
:101E400004C2938002D293A207B34005E556B407BB
:101E5000037573CDE595C395734004C2948002D297
:101E600094E54575F00284FF7E0090018012001E0B
:101E7000E075F00284FF7E00EF24CDF570E595C398
:101E800095705017A20CB34002D291A20DB340023C
:101E9000D292A20EB34002D2908006C291C292C2E8
:101EA00090E543C39406400302250CA2EDB3500312
:101EB00002250CC2EDE54360030220067E017F008F
:101EC000E5BE124204E5BD2FFF50010E900000EE6A
:101ED000F0A3EFF0900029E0B401177E0F7FFF9090
:101EE0000000E0FCA3E0FD120003900000EEF0A370
:101EF000EFF0900079E0B4025B900000E0FEA3E018
:101F0000FF90000AE0FCA3E0FDEDD39FEC9E400FA4
:101F1000900000E0F8A3E090000AC8F0A3C8F09099
:101F20000000E0FEA3E0FF90000CE0FCA3E0FDEF6A
:101F3000D39DEE9C400F900000E0F8A3E090000CD1
:101F4000C8F0A3C8F0900000E0FEA3E0FF74041204
:101F500041F68F44900079E07060900000E0FEA3AD
:101F6000E0FF90000AE0FCA3E0FDEFD39DEE9C4073
:101F70000D120003900000EEF0A3EFF08007900038
:101F800000E4F0A3F0900000E0FEA3E0FF74101264
:101F90004204900026E08E048F05FF1241E6900077
:101FA00000ECF0A3EDF07400D39D74019C40089008
:101FB0000001E0F54480037544FFE54475F00AA490
:101FC000FFAEF074198E048F05FF1241E68D45EDCA
:101FD0002532FFAE3150010E74011241F68F458556
:101FE0004532753100EFD39462400375456290002D
:101FF00072E064016006900066E06002800575434F
:1020000001800375BB17E543B4010280030220F68B
:102010007E017F00E5BE124204E5BD2FFF50010E98
:10202000900000EEF0A3EFF0900072E0B4017EE5C6
:102030003445336025AC33AD341DBDFF011C8F0228
:102040008E038C068D07903ECE12002EE493FE7414
:102050000193FFEFC39AEE9B400280057833124252
:102060002EAE33AF3474B3BE0025D39F4021900011
:1020700000E0FCA3E0FD0FBF00010E903ECE120079
:102080002EE493FE740193FFEDC39FEC9E4002800B
:1020900005783312003FAE33AF34E56B124204745F
:1020A000648E048F05FF1241E68D478033900066F1
:1020B000E0602D900000E0FEA3E0FFEFD39400EE7F
:1020C0009408400F900066E0B40104C2098002D277
:1020D00009800D900066E0B40104D2098002C209B3
:1020E000900072E064026006900066E0600575BBD7
:1020F000168003754302E543B4020280030221E423
:102100007E017F00E5BE124204E5BD2FFF50010EA7
:10211000900000EEF0A3EFF0900072E0B4027EE5D4
:102120003445336025AC33AD341DBDFF011C8F0237
:102130008E038C068D07903D6412002EE493FE748E
:102140000193FFEFC39AEE9B400280057833124261
:102150002EAE33AF3474B3BE0025D39F4021900020
:1021600000E0FCA3E0FD0FBF00010E903D641200F3
:102170002EE493FE740193FFEDC39FEC9E4002801A
:1021800005783312003FAE33AF34E56B124204746E
:10219000648E048F05FF1241E68D47803390006600
:1021A000E0602D900000E0FEA3E0FFEFD39400EE8E
:1021B0009408400F900066E0B40104C2098002D286
:1021C00009800D900066E0B40104D2098002C209C2
:1021D000900072E07003754700900066E07002C2E4
:1021E0000975BB1FE543B403457E017F00E5BE12C0
:1021F0004204E5BD2FFF50010E900000EEF0A3EF6A
:10220000F0740912420474E68E048F05FF1241E651
:102210008C418D42E54A2DFD50010C74018C068DD8
:10222000071241F68E418F4285424A75BB19E5433C
:10223000B4040280030223F47E017F00E5BE124253
:1022400004E5BD2FFF50010E900000EEF0A3EFF06B
:1022500074041241F68F4BE565B40102800302233A
:102260004F756C00756C00E56CD394074003022336
:1022700006E56C90004112421CE0D3954B501AE5E4
:102280006C90004112421CE0F404254BFEE56C907A
:10229000003712421CEEF08017E56C9000411242AC
:1022A0001CE0C3954BFEE56C90003712421CEEF02B
:1022B000E56CC394044009900084E0C3956C503BE6
:1022C000E56C6029E56C90003712421CFEE0FFEEE1
:1022D00090003FE0D39F4013E56C90003712421C02
:1022E000E090003FF0E56C900040F0800E900037E9
:1022F000E090003FF07400900040F0786C7401268C
:10230000F64003022267900040E0F4042408F556EA
:10231000E556D394054006E5B554FDF5B5E5586599
:1023200056602CE558D394054007E556C394064003
:10233000028005E55104F552855658E556C39404CC
:102340005007E55604F5578003855657755B00E541
:1023500065D394014061E54BD3946E4004D2108064
:1023600002C210755605E565B40205A210B340021D
:102370008003755607E565B40306A210B3B34002A7
:102380008003755607E5586556602CE558D39405CB
:102390004007E556C3940640028005E55104F55216
:1023A000855658E556C394045007E55604F5578002
:1023B00003855657755B00E55865566008E551047E
:1023C000F552855658E556B40708E5B54480F5B58D
:1023D0008006E5B5547FF5B5E55664066005E5561B
:1023E000B40808E5B54440F5B58006E5B554BFF539
:1023F000B575BB13E543B4050280030225087E01D1
:102400007F00E5BE124204E5BD2FFF50010E900093
:1024100000EEF0A3EFF074041241F68F46E564B4C9
:1024200002028003022505756C00756C00E56CD313
:10243000940340030224BCE56C90003312421CE07C
:10244000D39546501AE56C90003312421CE0F40418
:102450002546FEE56C90002D12421CEEF08017E53B
:102460006C90003312421CE0C39546FEE56C900070
:102470002D12421CEEF0E56C6029E56C90002D12E7
:10248000421CFEE0FFEE900031E0D39F4013E56C6C
:1024900090002D12421CE0900031F0E56C9000326B
:1024A000F0800E90002DE0900031F074009000322A
:1024B000F0786C740126F6400302242D900082E02F
:1024C0007043E52A45296036E559C39403500A90C4
:1024D0000032E004C3940340028007900032E0041D
:1024E000F559E559D39402400A900032E004D394A0
:1024F0000250028007900032E004F55980079000F6
:1025000032E004F55975BB180543D2ECE55FD3946E
:102510000450030226BB75CF01C293AE35AF3674AB
:1025200088D39F74139E4005A2A5B34014AE35AF67
:10253000367488D39F74139E4005A2A4B3400280D2
:1025400048783512003FAE35AF36EFB4883BEEB475
:102550001337A2A5B3500990004FE0D39551500214
:10256000800405518011A2A5B3500890004FE0658A
:102570005160028002D207A2A4B35007E551D39460
:1025800001500280041551C207A2A5B3B35006A2A0
:10259000A4B3B340028006753600753500E5516579
:1025A00052700302265FE55175F040A4FFAEF09033
:1025B000032212001EE030E003D38001C3B34008C1
:1025C000E5B54410F5B58006E5B554EFF5B5E55130
:1025D00075F040A4FFAEF090032312001EE030E03F
:1025E00003D38001C3B34008E5B54420F5B58006A8
:1025F000E5B554DFF5B5E55175F040A4FFAEF090B8
:10260000032412001EE030E003D38001C39287E56B
:102610005175F040A4FFAEF090032512001EE0308B
:10262000E003D38001C3920CE55175F040A4FFAEE6
:10263000F090032612001EE030E003D38001C39225
:102640000DE55175F040A4FFAEF090032712001E77
:10265000E030E003D38001C3920EC294855152A2B0
:102660000740057573CD80037573FFE595C39573BA
:102670004004C2948002D294E54575F00284FF7E46
:102680000090018012001EE075F00284FF7E00EFD2
:1026900024CDF570E595C395705017A20CB3400298
:1026A000D291A20DB34002D292A20EB34002D290B8
:1026B0008006C291C292C290022516AE25AF26EFC7
:1026C000D39420EE944E50030227AA120471C28EB6
:1026D000758D00758B00754C00D28EC20775720027
:1026E0007571007573CD75510575240075230075DE
:1026F0005400755B00C296900059E06004D295804A
:1027000002C29590004AE0B40104D2978002C297B9
:10271000900049E0B40104D2A08002C2A0A209B393
:102720004004D2A28002C2A290006BE0601812386E
:1027300083A200B34008E5B54408F5B58006E5B5C9
:1027400054F7F5B58002C20090006EE060101239B7
:10275000D8A202B34004D2A18002C2A18002C2A1C9
:1027600090000E74FDF0A374E8F0E543B406037521
:102770004300900025E4F0752600752500758D0056
:10278000758B00754C00900024E0C39403500890B2
:102790000024E004F080067403900024F0900024EC
:1027A000E0B40306E5B554FEF5B5AE27AF28EFD388
:1027B0009410EE9427401CC2CA75CD0075CC0075EC
:1027C0002800752700D2CA754E00752A00752900A9
:0627D000755500020AC865
:103B8A00000001000132016401960196020002124E
:103B9A0002240200020003000340038003C0040061
:103BAA000440048004C00500060006000600060062
:103BBA00060006000600060000FF013101630195B8
:103BCA0001FF01FF0211022302FF02FF02FF033F6E
:103BDA00037F03BF03FF043F047F04BF04FF05FF05
:103BEA0006FF06FF06FF06FF06FF06FF06FF06FFA3
:103BFA000FAA0FA50F9F0F9A0F940F8D0F870F8093
:103C0A000F780F710F680F600F570F4E0F450F3B5C
:103C1A000F300F250F1A0F0E0F020EF50EE80EDBEE
:103C2A000ECC0EBE0EAE0E9F0E8E0E7D0E6C0E5A72
:103C3A000E470E340E200E0C0DF70DE20DCB0DB50E
:103C4A000D9D0D850D6D0D540D3A0D200D050CE9D8
:103C5A000CCE0CB10C940C760C580C3A0C1B0BFBCA
:103C6A000BDB0BBB0B9A0B790B570B350B130AF1BA
:103C7A000ACE0AAB0A870A640A400A1C09F809D460
:103C8A0009B0098C09670943091F08FB08D608B25D
:103C9A00088E086A0846082307FF07DC07B9079653
:103CAA0007730751072F070D06EC06CA06AA0689ED
:103CBA0006690649062A060A05EC05CD05B00592ED
:103CCA0005750558053C0520050504EA04CF04B529
:103CDA00049C04820469045104390422040B03F489
:103CEA0003DE03C803B2039D038903750361034D11
:103CFA00033B03280316030402F202E102D102C0C5
:103D0A0002B002A0029102820273026502570249BE
:103D1A00023C022F02220216020901FD01F201E60B
:103D2A0001DB01D001C601BB01B101A7019D0194CC
:103D3A00018B01820179017001680160015801500B
:103D4A000148014101390132012B0125011E0118E7
:103D5A000111010B010500FF00FA0FA60FA00F9930
:103D6A000F920F8B0F840F7C0F740F6B0F620F581B
:103D7A000F4E0F430F380F2C0F1F0F120F050EF7A0
:103D8A000EE80ED80EC80EB70EA50E930E800E6C56
:103D9A000E580E420E2C0E150DFD0DE40DCB0DB175
:103DAA000D950D790D5D0D3F0D200D010CE10CC037
:103DBA000C9E0C7C0C590C350C100BEA0BC40B9E98
:103DCA000B760B4F0B260AFD0AD40AAA0A800A555B
:103DDA000A2A09FF09D409A8097C0950092508F902
:103DEA0008CD08A10875084A081E07F307C8079DE9
:103DFA0007730749072006F706CE06A6067E06576A
:103E0A000630060A05E405BF059B05770554053209
:103E1A00051004EF04CE04AE048F04710453043574
:103E2A00041903FD03E203C703AD0394037B036391
:103E3A00034B0334031E030802F302DE02CA02B66E
:103E4A0002A30291027F026D025C024C023C022C28
:103E5A00021D020E020001F201E401D701CA01BEED
:103E6A0001B101A6019A018F0185017A01700166EB
:103E7A00015D0153014A0141013901310129012141
:103E8A0001190112010B010400FD00F700F000EA1C
:103E9A0000E400DE00D900D300CE00C900C400BF90
:103EAA0000BA00B500B100AD00A800A400A0009CB3
:103EBA00009900950091008E008A00870084008195
:043ECA00007E007BFB
:1027F700751A00751900AE19AF1AAC17AD18EDC3ED
:102807009FEC9E401674FF1241D675CF01781A745B
:102817000126F6500418E436F650DB22900786E4CA
:10282700F0A3F0751000750F00751300751400C242
:1028370011D21222C2AF75D900758F0375B7A5756E
:10284700B7F190F800E4F0758F0175B7A575B7F18A
:10285700E50890F800F075B7A575B7F190F801E4B1
:10286700F075B7A575B7F190079DE090F802F07580
:10287700B7A575B7F19007A1E090F803F075B7A574
:1028870075B7F190079EE090F804F075B7A575B796
:10289700F190079FE090F805F075B7A575B7F1902F
:1028A70007A0E090F806F075B7A575B7F19007A2F5
:1028B700E090F807F0758F0075D940D2AF229007E6
:1028C70088E0B4AB61C2AF75D90075B62275F52241
:1028D700758F0375B7A575B7F1740090F600F0759D
:1028E7008F01750A00750900AE09AF0A7413BE009F
:1028F700279F402475B7A575B7F190078912001E69
:10290700E0FC90F60012001EECF0780A740126F63F
:10291700500418E436F650D0758F0075F51175B66A
:102927002075D940D2AF22C2AF75D90075F522758F
:102937000A00750900AE09AF0A7413BE00229F4052
:102947001F90F60012001EE493FC90078912001EE8
:10295700ECF0780A740126F6500418E436F650D5E0
:1029670075F51175D940D2AF22900788E0B4AA0255
:102977008003022AADC2AF75D90075B62275F5225C
:10298700758F0375B7A575B7F1740090EE00F075F4
:10299700B7A575B7F1740090F000F075B7A575B7D6
:1029A700F1740090F200F075B7A575B7F174009057
:1029B700F400F0758F01750A00750900AE09AF0ABA
:1029C70074FFC39F74019E402475B7A575B7F19036
:1029D700004E12001EE0FC90EE0012001EECF07894
:1029E7000A740126F6500418E436F650CF750A002B
:1029F700750900AE09AF0A74FFC39F74019E402496
:102A070075B7A575B7F190024E12001EE0FC90F065
:102A17000012001EECF0780A740126F6500418E440
:102A270036F650CF750A00750900AE09AF0A74FF74
:102A3700C39F74019E402475B7A575B7F190044EE6
:102A470012001EE0FC90F20012001EECF0780A74EF
:102A57000126F6500418E436F650CF750A007509BA
:102A670000AE09AF0A74FFC39F74019E402475B777
:102A7700A575B7F190064E12001EE0FC90F4001207
:102A8700001EECF0780A740126F6500418E436F6B6
:102A970050CF758F0075F51175B62075D940D2AF37
:102AA700743A90074EF022900788E0B4AA02800398
:102AB700022BEBC2AF75D90075B62275F522758F5B
:102AC7000375B7A575B7F1740090E600F075B7A563
:102AD70075B7F1740090E800F075B7A575B7F17494
:102AE7000090EA00F075B7A575B7F1740090EC0097
:102AF700F0758F01750A00750900AE09AF0A74FFFA
:102B0700C39F74019E402475B7A575B7F190004E19
:102B170012001EE0FC90E60012001EECF0780A742A
:102B27000126F6500418E436F650CF750A007509E9
:102B370000AE09AF0A74FFC39F74019E402475B7A6
:102B4700A575B7F190024E12001EE0FC90E8001246
:102B5700001EECF0780A740126F6500418E436F6E5
:102B670050CF750A00750900AE09AF0A74FFC39FFD
:102B770074019E402475B7A575B7F190044E1200F5
:102B87001EE0FC90EA0012001EECF0780A740126A1
:102B9700F6500418E436F650CF750A00750900AEF2
:102BA70009AF0A74FFC39F74019E402475B7A575CA
:102BB700B7F190064E12001EE0FC90EC0012001ECA
:102BC700ECF0780A740126F6500418E436F650CF74
:102BD700758F0075F51175B62075D940D2AF743A67
:102BE70090074EF022900788E0B4AA028003022DD6
:102BF70029C2AF75D90075B62275F522758F037591
:102C0700B7A575B7F1740090DE00F075B7A575B775
:102C1700F1740090E000F075B7A575B7F1740090F6
:102C2700E200F075B7A575B7F1740090E400F07590
:102C37008F01750A00750900AE09AF0A74FFC39FBB
:102C470074019E402475B7A575B7F190004E120028
:102C57001EE0FC90DE0012001EECF0780A740126DC
:102C6700F6500418E436F650CF750A00750900AE21
:102C770009AF0A74FFC39F74019E402475B7A575F9
:102C8700B7F190024E12001EE0FC90E00012001E09
:102C9700ECF0780A740126F6500418E436F650CFA3
:102CA700750A00750900AE09AF0A74FFC39F740166
:102CB7009E402475B7A575B7F190044E12001EE02B
:102CC700FC90E20012001EECF0780A740126F65020
:102CD7000418E436F650CF750A00750900AE09AF3F
:102CE7000A74FFC39F74019E402475B7A575B7F199
:102CF70090064E12001EE0FC90E40012001EECF05D
:102D0700780A740126F6500418E436F650CF758F0A
:102D17000075F51175B62075D940D2AF743A900792
:102D27004EF022900788E0B4AA028003022E67C201
:102D3700AF75D90075B62275F522758F0375B7A5DE
:102D470075B7F1740090D600F075B7A575B7F17433
:102D57000090D800F075B7A575B7F1740090DA0048
:102D6700F075B7A575B7F1740090DC00F0758F01A9
:102D7700750A00750900AE09AF0A74FFC39F740195
:102D87009E402475B7A575B7F190004E12001EE05E
:102D9700FC90D60012001EECF0780A740126F6505B
:102DA7000418E436F650CF750A00750900AE09AF6E
:102DB7000A74FFC39F74019E402475B7A575B7F1C8
:102DC70090024E12001EE0FC90D80012001EECF09C
:102DD700780A740126F6500418E436F650CF750ABF
:102DE70000750900AE09AF0A74FFC39F74019E40C6
:102DF7002475B7A575B7F190044E12001EE0FC903C
:102E0700DA0012001EECF0780A740126F650041856
:102E1700E436F650CF750A00750900AE09AF0A749B
:102E2700FFC39F74019E402475B7A575B7F190063F
:102E37004E12001EE0FC90DC0012001EECF0780A37
:102E4700740126F6500418E436F650CF758F0075D6
:102E5700F51175B62075D940D2AF743A90074EF088
:102E670022C2AF75D90075F522750A00750900AE43
:102E770009AF0A74FFC39F74019E401F90EE0012B2
:102E8700001EE493FC90004E12001EECF0780A74CA
:102E97000126F6500418E436F650D4750A00750971
:102EA70000AE09AF0A74FFC39F74019E401F90F0E4
:102EB7000012001EE493FC90024E12001EECF07804
:102EC7000A740126F6500418E436F650D4750A0041
:102ED700750900AE09AF0A74FFC39F74019E401FB6
:102EE70090F20012001EE493FC90044E12001EECB8
:102EF700F0780A740126F6500418E436F650D475B3
:102F07000A00750900AE09AF0A74FFC39F74019EDA
:102F1700401F90F40012001EE493FC90064E12002E
:102F27001EECF0780A740126F6500418E436F650C1
:102F3700D475F51175D940D2AF22C2AF75D90075D6
:102F4700F522750A00750900AE09AF0A74FFC39F21
:102F570074019E401F90E60012001EE493FC90004F
:102F67004E12001EECF0780A740126F6500418E49D
:102F770036F650D4750A00750900AE09AF0A74FF1A
:102F8700C39F74019E401F90E80012001EE493FC4B
:102F970090024E12001EECF0780A740126F65004D7
:102FA70018E436F650D4750A00750900AE09AF0A61
:102FB70074FFC39F74019E401F90EA0012001EE435
:102FC70093FC90044E12001EECF0780A740126F66A
:102FD700500418E436F650D4750A00750900AE0996
:102FE700AF0A74FFC39F74019E401F90EC0012004C
:102FF7001EE493FC90064E12001EECF0780A740152
:1030070026F6500418E436F650D475F51175D940F4
:10301700D2AF22C2AF75D90075F522750A007509BE
:1030270000AE09AF0A74FFC39F74019E401F90DE74
:103037000012001EE493FC90004E12001EECF07884
:103047000A740126F6500418E436F650D4750A00BF
:10305700750900AE09AF0A74FFC39F74019E401F34
:1030670090E00012001EE493FC90024E12001EEC4A
:10307700F0780A740126F6500418E436F650D47531
:103087000A00750900AE09AF0A74FFC39F74019E59
:10309700401F90E20012001EE493FC90044E1200C1
:1030A7001EECF0780A740126F6500418E436F65040
:1030B700D4750A00750900AE09AF0A74FFC39F747F
:1030C700019E401F90E40012001EE493FC90064E00
:1030D70012001EECF0780A740126F6500418E43644
:1030E700F650D475F51175D940D2AF22C2AF75D954
:1030F7000075F522750A00750900AE09AF0A74FF5D
:10310700C39F74019E401F90D60012001EE493FCDB
:1031170090004E12001EECF0780A740126F6500457
:1031270018E436F650D4750A00750900AE09AF0ADF
:1031370074FFC39F74019E401F90D80012001EE4C5
:1031470093FC90024E12001EECF0780A740126F6EA
:10315700500418E436F650D4750A00750900AE0914
:10316700AF0A74FFC39F74019E401F90DA001200DC
:103177001EE493FC90044E12001EECF0780A7401D2
:1031870026F6500418E436F650D4750A007509007F
:10319700AE09AF0A74FFC39F74019E401F90DC0005
:1031A70012001EE493FC90064E12001EECF0780A03
:1031B700740126F6500418E436F650D475F51175E7
:1031C700D940D2AF22E51464046006E59964FF6034
:1031D700028031A2114004D2118027E514600874DF
:1031E700E62514900023F0E513600874F02513908A
:1031F7000023F0E514B4010280FE75140075130076
:10320700C2118002C211E514903B2DF8282873756E
:103217001400E599B4FF03751301E599B4FE03752E
:103227001302E599B4FD03751303E599B4FC03751F
:103237001304E599B4FA03751305E599B4FB06750C
:103247001401120471E599B4F90675140412047196
:10325700E599D394E54007E599C394F040028016B9
:103267008599157514027E017F00E515C394E61252
:1032770042048E0D8F0E900786E4F0A3F0E599D3F4
:1032870094C44007E599C394E640028028859915C0
:1032970075140374E5C39515F50E750D00AE0DAFE6
:1032A7000E903B8A12002EE493F8740193900786E0
:1032B700C8F0A3C8F0D299023741900786E0FEA371
:1032C700E0FFEFC39400EE94054009EFD394FFEEBF
:1032D70094064013900786E0FEA3E0FF90004E128D
:1032E700001EE599F0800385996D90078612000E00
:1032F700900786E0FEA3E0FFEFB40106EEB40702F5
:10330700800302354E90074EE0B43C02800302353D
:103317004E75FFA0A20AB35005A20BB340030234B7
:1033270041C29C90007AE090078CF0900057E090A3
:10333700078DF0900062E090078EF0900063E090B8
:10334700078FF0900074E0900790F090007CE09079
:103357000791F090007DE0900792F0900080E09058
:103367000793F0900081E0900794F090013AE09085
:103377000795F090013BE0900796F090013CE090B4
:103387000797F0900090E0900798F0900091E090F8
:103397000799F0900092E090079AF0900093E090E0
:1033A700079BF0900094E090079CF0900095E090C8
:1033B700079DF0900096E090079EF0900097E090B0
:1033C700079FF0900099E09007A0F090009AE09096
:1033D70007A1F090009BE09007A2F090009CE0907E
:1033E70007A3F07400900082F012008F74AB90076F
:0D33F70088F01228C574AA900788F0E559E7
:063B2D000232160232C153
:10340400903B4EF82828738012122970800D122ADE
:0B341400AE8008122BEC8003122D2A62
:0F3B4E0002340B02340D02341202341702341CFD
:10341F00900788E4F090013AE0700C90013BE07067
:10342F000690013CE060028004C20A8002D20A02C8
:10343F003543C29C900078E0900789F090005EE0E1
:10344F0090078AF090005FE090078BF090007AE091
:10345F0090078CF0900057E090078DF0900062E09D
:10346F0090078EF0900063E090078FF0900074E06B
:10347F00900790F090007CE0900791F090007DE035
:10348F00900792F0900080E0900793F0900081E019
:10349F00900794F090013AE0900795F090013BE08F
:1034AF00900796F090013CE0900797F0900090E025
:1034BF00900798F0900091E0900799F0900092E0BB
:1034CF0090079AF0900093E090079BF0900094E0A3
:1034DF0090079CF0900095E090079DF0900096E08B
:1034EF0090079EF0900097E090079FF0900099E072
:1034FF009007A0F090009AE09007A1F090009BE059
:10350F009007A2F090009CE09007A3F07400900049
:10351F0082F074AB900788F01228C574AA900788C0
:10352F00F0122970122AAE122BEC122D2AD29C7592
:10353F0099FB80FED29C7514007513007599FB02E0
:10354F003741900786E0FEA3E0FFEF4E70068599A6
:10355F0010750F00900786E0FEA3E0FF74016F4E19
:10356F00701BAC0FAD10AA0DAB0EED2BFBEC3AFAA6
:10357F008A068B0790004E12001EE599F090078681
:10358F0012000E900786E0FEA3E0FF74026F4E70EC
:10359F000C12008F851599751400751300023741B1
:1035AF00900786E0FEA3E0FF90004E12001EE59903
:1035BF00F090078612000E900786E0FEA3E0FFACA6
:1035CF000DAD0E8F028E038C068D07903BC212003D
:1035DF002EE493F9740193FEEAD39EEB994009858B
:1035EF001599751400751300023741900786E0FE98
:1035FF00A3E0FF90004E12001EE599F0900786128F
:10360F00000E900786E0FEA3E0FFEFB40006EEB4D5
:10361F000102800302374175FFA090001CE0D39494
:10362F00C7400B90001CE0C394C8F516801A900099
:10363F001CE0D39463400B90001CE0C39464F51618
:10364F00800690001CE0F516E51675F002A4FFAE9B
:10365F00F08F6CEF90004E12421CEFFCE0FDEC90EF
:10366F00005112421CEDFCE0FDEC2DB5160280035B
:10367F000237330FEF90004E12421CE56CFFE0FC57
:10368F00EF90005212421CECFFE0FCEFC39CB5160A
:10369F00028003023733E56C90005012421CE56C38
:1036AF00FFE0FCEF90005312421CECFFE0FCEF2C0C
:1036BF00B51671E56C90005412421CE0C39516903C
:1036CF00079DF0E56C90005512421CE0C3951690D3
:1036DF00079EF0E56C90005812421CE0C3951690BF
:1036EF00079FF0E56C90005912421CE0C3951690AD
:1036FF0007A0F0E56C90005A12421CE0C39516909B
:10370F0007A1F0E56C90005B12421CE0C395169088
:10371F0007A2F012283B7599F975186475170012F6
:10372F0027F780FE7599FF7518647517001227F734
:02373F0080FE0A
:093B33000235510235AF0235FAEA
:1037410022E513903B3CF8282873023882900786C3
:10375100E0FEA3E0FF90001212001EE0F599900731
:103761008612000E900786E0FEA3E0FF74116F4EF3
:1037710070037513000238828563990238829007BD
:1037810086E0FEA3E0FF90004E12001EE0F599EFE7
:10379100B40107EEB4070375130090078612000EFB
:0737A100023882900787E067
:0F3B3C0002374B02374E02377902377F0237A428
:1037A800903B5DF8282873852499023877852A99F3
:1037B80002387785449902387785479902387785A2
:1037C8005199023877856199023877855699023878
:1037D80077855999023877756F00900069E070060F
:1037E800900068E060028016A2A44006E56F4404D9
:1037F800F56FA2A54006E56F4402F56F801A9000A8
:103808004AE0B40106E56F4410F56F900049E0B452
:103818000106E56F4420F56FA207B34006E56F4443
:1038280001F56FA209B34006E56F4408F56F856F8F
:1038380099803CA212B340077599FAC2128017A268
:103848000FB3400575990F800B900023E0F5999010
:103858000023E4F0C20F80178542998012854B99A6
:0F386800800D85469980087599FC8003751300C3
:103B5D000237AF0237B50237BB0237C10237C70292
:103B6D0037CD0237D30237D90237DF02383B02385F
:0D3B7D006002386502386A02386F02387441
:0B38770090078612000E80031200482C
:033B4B0002387FBE
:103882002290006BE0B4010385241190006BE0B438
:103892000203852A1190006BE0B403038544119062
:1038A200006BE0B4040385471190006BE0B405039C
:1038B20085511190006BE0B4060385561190006BA0
:1038C200E0B4070385591190006CE0FE90006DE0B2
:1038D200C39E500302395990006BE0D39404402CEC
:1038E20090006CE0D39511500990006DE0C39511E2
:1038F20050028002D20090006CE0D39511500990E2
:10390200006DE0C395115002C200804990006BE047
:10391200B4041890006DE0C395115002D2009000DB
:103922006CE0D395114002C200802A90006CE0C383
:103932009511500990006DE0D3951150028002D28A
:103942000090006CE0D39511500990006DE0C39592
:10395200115002C200807E90006BE0D39404402C90
:1039620090006CE0C39511400990006DE0D3951171
:1039720040028002C20090006CE0C39511400990A1
:10398200006DE0D395114002D200804990006BE0B7
:10399200B4041890006CE0C395115002C20090006C
:1039A2006DE0D395114002D200802A90006CE0C3F2
:1039B2009511400990006DE0D395114002D200901C
:1039C200006CE0D39511400990006DE0C395114061
:1039D200028002C2002290006EE0B401038524112D
:1039E20090006EE0B40203852A1190006EE0B403E9
:1039F2000385441190006EE0B404038547119000E2
:103A02006EE0B4050385511190006EE0B4060385A3
:103A1200561190006EE0B4070385591190006FE0D3
:103A2200FE900070E0C39E5003023AAE90006EE03A
:103A3200D39404402C90006FE0D39511500990006C
:103A420070E0C3951150028002D20290006FE0D361
:103A520095115009900070E0C395115002C2028086
:103A62004990006EE0B40418900070E0C3951150C4
:103A720002D20290006FE0D395114002C202802A66
:103A820090006FE0C395115009900070E0D395113A
:103A920050028002D20290006FE0D395115009903B
:103AA2000070E0C395115002C202807E90006EE069
:103AB200D39404402C90006FE0C39511400990000C
:103AC20070E0D3951140028002C20290006FE0C301
:103AD20095114009900070E0D395114002D2028006
:103AE2004990006EE0B4041890006FE0C395115045
:103AF20002C202900070E0D395114002D202802AE5
:103B020090006FE0C395114009900070E0D39511C9
:103B12004002D20290006FE0D395114009900070EC
:0B3B2200E0C3951140028002C20222A5
:09421C002582F58250020583227F
:10002E00EF2F500205832582F582E5833E2EF58360
:01003E00229F
:08000300C3EF9DFFEE9CFE22FD
:08003F000806B60002180622B3
:0D000E00A3E004F07006124212E004F0229C
:08422E000816B6FF0218162263
:0E41F600048007C3CE13CECF13CFD5E0F62240
:1040A400BC000FBE0008ED8FF084FFADF022E4FEEB
:1040B400FF22BE000DEF60FE54F0606F20E70302A4
:1040C400415AEAC0E0EBC0E078017A0075F001EEF5
:1040D40020E710EF25E0FFEE33FE0AC5F023C5F01C
:1040E40030E7F0EA5407F9096A7A007B00600108B6
:1040F400C3EC9E40167004ED9F4010ED9FFDEC9EB6
:10410400FCE5F0CA4ACA03F5F08005E5F003F5F0D2
:10411400C3EE13FEEF13FFD9D77908CACBCAD8D0A0
:10412400EAFEEBFFD0E0FBD0E0FA22EC8FF084FC57
:10413400ED54F045F0C48FF084FEEDC454F045F026
:10414400C48FF084FDEEC4FE54F02DFFEE540F3CFA
:10415400FEADF07C0022790078008FF0EC7E082020
:10416400E70DC3CD33CD33C933C9C833C8DEF084BA
:1041740049F9E5F08FF0BE00E6FD7C00E9FFE8FEBA
:014184002218
:0E420400F88FF0A4FFE5F0CE88F0A42EFE2285
:1041D600600D782B0241E0007830D8FED5E0F82259
:1041E600EEC0E07E001240A4EFFDEEFCD0E0FE2221
:03000B000241852A
:03001B000241A0FF
:03002B000241BBD4
:0300000002422594
:0942250075817475D00002064594
:0B001E00E5822FF582E5833EF583228A
:0A4212000582D58202158315822271
:10418500C0E0C0F0C083C082C0D075D00012063A2E
:10419500D0D0D082D083D0F0D0E032C0E0C0F0C023
:1041A50083C082C0D075D00012063DD0D0D082D059
:1041B50083D0F0D0E032C0E0C0F0C083C082C0D070
:1041C50075D000120640D0D0D082D083D0F0D0E098
:0141D50032B7
:00000001FF
